:100000000EC020C01FC01EC01DC01CC01BC01AC017
:1000100019C018C017C016C015C014C013C01124D1
:100020001FBECFE5D2E0DEBFCDBF10E0A0E6B0E05E
:10003000EEECF1E002C005900D92A236B107D9F7BF
:1000400002D0C3C0DDCFF89487B3836187BB83EA56
:100050008ABD91E093BF8FEF89BD88BD90BF90E6C8
:100060009CBD8BBD8DBD78949FE730E888BD1BBCDF
:1000700019BC2FEF49E658E1215040405040E1F7CC
:1000800000C000008093600020916000222389F06E
:100090002150209360002F3708F028BD2091600088
:1000A00020952BBDEFE4F3EC3197F1F700C0000091
:1000B000EBCF98BD8BBD19BCFFEF29E648E1F150AD
:1000C00020404040E1F700C0000010926000209105
:1000D000600027FD15C041E0420F40936000592F9A
:1000E000521B58BD2091600020952BBD20916000CF
:1000F00029BDEFE4F3EC3197F1F700C00000E7CF42
:10010000209160002F3F59F02F5F2093600029BDA0
:10011000EFE4F3EC3197F1F700C00000F1CF18BC29
:100120009BBD29BDFFEF29E648E1F150204040404A
:10013000E1F700C00000109260002091600027FDF0
:1001400010C02F5F2093600028BD20916000532FC6
:10015000521B5BBDEFE4F3EC3197F1F700C00000F8
:10016000ECCF98BD1BBC89BDFFEF29E648E1F150FB
:1001700020404040E1F700C0000010926000209154
:10018000600027FD11C041E0420F409360002058FD
:1001900028BD20916000209529BDEFE4F3EC319754
:1001A000F1F700C00000EBCF209160002F3F09F471
:1001B0005DCF2F5F20936000209529BDEFE4F3EC25
:0E01C0003197F1F700C00000EFCFF894FFCFA9
:0201CE00FF0030
:00000001FF
